BL51 BANKED LINKER/LOCATER V6.00                                                        01/16/2018  10:49:12  PAGE 1


BL51 BANKED LINKER/LOCATER V6.00, INVOKED BY:
C:\KEIL\C51\BIN\BL51.EXE main.obj TO MA82G5Dxx RAMSIZE (256)


MEMORY MODEL: SMALL


INPUT MODULES INCLUDED:
  main.obj (MAIN)
  C:\KEIL\C51\LIB\C51S.LIB (?C_STARTUP)


LINK MAP OF MODULE:  MA82G5Dxx (MAIN)


            TYPE    BASE      LENGTH    RELOCATION   SEGMENT NAME
            -----------------------------------------------------

            * * * * * * *   D A T A   M E M O R Y   * * * * * * *
            REG     0000H     0008H     ABSOLUTE     "REG BANK 0"
            DATA    0008H     0002H     UNIT         ?DT?MAIN
            IDATA   000AH     0001H     UNIT         ?STACK

            * * * * * * *   C O D E   M E M O R Y   * * * * * * *
            CODE    0000H     0003H     ABSOLUTE     
            CODE    0003H     001EH     UNIT         ?PR?MAIN?MAIN
            CODE    0021H     0016H     UNIT         ?PR?_PAGEP_WRITE?MAIN
            CODE    0037H     0016H     UNIT         ?PR?_PAGEP_READ?MAIN
            CODE    004DH     0004H     UNIT         ?PR?START_WDT?MAIN
                    0051H     0002H                  *** GAP ***
            CODE    0053H     0003H     ABSOLUTE     
            CODE    0056H     000DH     UNIT         ?PR?INITIAL_WDT?MAIN
            CODE    0063H     000CH     UNIT         ?C_C51STARTUP
            CODE    006FH     000AH     UNIT         ?PR?STOP_WDT?MAIN
            CODE    0079H     0007H     UNIT         ?PR?INT_SYS?MAIN



OVERLAY MAP OF MODULE:   MA82G5Dxx (MAIN)


SEGMENT
  +--> CALLED SEGMENT
---------------------
?C_C51STARTUP
  +--> ?PR?MAIN?MAIN

?PR?MAIN?MAIN
  +--> ?PR?INITIAL_WDT?MAIN

?PR?INITIAL_WDT?MAIN
  +--> ?PR?START_WDT?MAIN



SYMBOL TABLE OF MODULE:  MA82G5Dxx (MAIN)

  VALUE           TYPE          NAME
BL51 BANKED LINKER/LOCATER V6.00                                                      01/16/2018  10:49:12  PAGE 2


  ----------------------------------

  -------         MODULE        MAIN
  C:0000H         SYMBOL        _ICE_DUMMY_
  D:0090H         PUBLIC        P1
  D:00A0H         PUBLIC        P2
  D:00E7H         PUBLIC        ISPCR
  D:00C0H         PUBLIC        XICON
  D:00B0H         PUBLIC        P3
  D:00E8H         PUBLIC        P4
  D:00ADH         PUBLIC        EIE1
  D:00F8H         PUBLIC        P6
  D:00E1H         PUBLIC        WDTCR
  B:00A8H.7       PUBLIC        EA
  C:0037H         PUBLIC        _PageP_Read
  D:00A8H         PUBLIC        IE
  D:00B8H         PUBLIC        IP0L
  C:0021H         PUBLIC        _PageP_Write
  C:0056H         PUBLIC        Initial_WDT
  D:00D8H         PUBLIC        CCON
  C:0003H         PUBLIC        main
  D:00E6H         PUBLIC        SCMD
  D:008EH         PUBLIC        SFIE
  D:00E3H         PUBLIC        IFADRH
  D:00E5H         PUBLIC        IFMT
  B:00B0H.0       PUBLIC        P30
  D:00E4H         PUBLIC        IFADRL
  D:0088H         PUBLIC        TCON
  D:0008H         PUBLIC        ESF_Flag
  C:0079H         PUBLIC        INT_SYS
  D:0009H         PUBLIC        tmp
  D:00E2H         PUBLIC        IFD
  C:004DH         PUBLIC        Start_WDT
  D:0087H         PUBLIC        PCON0
  D:0097H         PUBLIC        PCON1
  D:0098H         PUBLIC        S0CON
  D:00C8H         PUBLIC        T2CON
  C:006FH         PUBLIC        Stop_WDT
  D:00D0H         PUBLIC        PSW
  -------         PROC          _PAGEP_WRITE
  D:0007H         SYMBOL        Addr
  D:0005H         SYMBOL        Data
  C:0021H         LINE#         26
  C:0021H         LINE#         27
  C:0021H         LINE#         28
  C:0024H         LINE#         29
  C:0026H         LINE#         30
  C:0028H         LINE#         31
  C:002BH         LINE#         32
  C:002EH         LINE#         33
  C:0031H         LINE#         34
  C:0034H         LINE#         35
  C:0036H         LINE#         36
  -------         ENDPROC       _PAGEP_WRITE
  -------         PROC          _PAGEP_READ
  D:0007H         SYMBOL        Addr
  -------         DO            
BL51 BANKED LINKER/LOCATER V6.00                                                      01/16/2018  10:49:12  PAGE 3


  D:0007H         SYMBOL        Data
  -------         ENDDO         
  C:0037H         LINE#         38
  C:0037H         LINE#         39
  C:0037H         LINE#         42
  C:003AH         LINE#         43
  C:003CH         LINE#         44
  C:003FH         LINE#         45
  C:0042H         LINE#         46
  C:0045H         LINE#         47
  C:0048H         LINE#         48
  C:004AH         LINE#         49
  C:004CH         LINE#         51
  C:004CH         LINE#         52
  -------         ENDPROC       _PAGEP_READ
  -------         PROC          STOP_WDT
  C:006FH         LINE#         56
  C:006FH         LINE#         57
  C:006FH         LINE#         58
  C:0072H         LINE#         59
  -------         ENDPROC       STOP_WDT
  -------         PROC          START_WDT
  C:004DH         LINE#         62
  C:004DH         LINE#         63
  C:004DH         LINE#         64
  C:0050H         LINE#         65
  -------         ENDPROC       START_WDT
  -------         PROC          INITIAL_WDT
  C:0056H         LINE#         67
  C:0056H         LINE#         68
  C:0056H         LINE#         69
  C:0059H         LINE#         70
  C:005CH         LINE#         71
  C:005FH         LINE#         72
  C:0062H         LINE#         73
  -------         ENDPROC       INITIAL_WDT
  -------         PROC          INT_SYS
  C:0079H         LINE#         75
  C:0079H         LINE#         77
  C:007CH         LINE#         78
  C:007FH         LINE#         80
  -------         ENDPROC       INT_SYS
  -------         PROC          MAIN
  C:0003H         LINE#         82
  C:0003H         LINE#         83
  C:0003H         LINE#         84
  C:0006H         LINE#         85
  C:0008H         LINE#         87
  C:000BH         LINE#         88
  C:000DH         LINE#         89
  C:000FH         LINE#         90
  C:0011H         LINE#         91
  C:0013H         LINE#         94
  C:0013H         LINE#         95
  C:0013H         LINE#         96
  C:0017H         LINE#         97
  C:0017H         LINE#         98
BL51 BANKED LINKER/LOCATER V6.00                                                      01/16/2018  10:49:12  PAGE 4


  C:001AH         LINE#         100
  C:001CH         LINE#         101
  C:001CH         LINE#         103
  C:001FH         LINE#         104
  -------         ENDPROC       MAIN
  -------         ENDMOD        MAIN

*** WARNING L16: UNCALLED SEGMENT, IGNORED FOR OVERLAY PROCESS
    SEGMENT: ?PR?_PAGEP_READ?MAIN

*** WARNING L16: UNCALLED SEGMENT, IGNORED FOR OVERLAY PROCESS
    SEGMENT: ?PR?STOP_WDT?MAIN

Program Size: data=11.0 xdata=0 code=126
LINK/LOCATE RUN COMPLETE.  2 WARNING(S),  0 ERROR(S)
